:041800000CEF0CF0ED
:10180800FACF23F0FBCF24F0E9CF25F053ED17F002
:0C181800D5EF19F0020E38EC1CF01200A5
:021826001700A9
:1022FA0001FC03020104FC0328C408F51200010EC4
:10230A0079EC1BF01200020E79EC1BF0120000D0DF
:10231A00A6B2FED71200D6CF03F0D7CF04F003C07F
:10232A0001F004C002F01200D6CF62F0D7CF63F0FA
:10233A0062C060F063C061F0120001C0A9FFA69CF0
:10234A00A69EA68000F000F0A85000D0120060C03F
:10235A00A9FFA69CA69EA68000F000F0A85000D077
:10236A0012000001606F010E0001F16F60C0F0F011
:10237A000201005100D01200016E01507F0BD56E90
:10238A00000ED76E000ED66EF29401AE02D0F28A1B
:10239A0001D0F29AD58E1200000E026E000E016E66
:1023AA00A2EC11F00001E26F040E0001E26504D014
:1023BA00000E0001E26F00D012000001E251050D8B
:1023CA00500EF3240001616F7F0EF4200001626F4A
:1023DA00050E0001636F33EC16F012000001E7519D
:1023EA00040D7D0EF3240001616F7F0EF4200001BD
:1023FA00626F040E0001636F33EC16F012000001E5
:10240A00E951050D910EF3240001616F7F0EF4204E
:10241A000001626F050E0001636F33EC16F01200C3
:10242A000001ED51060DAE0EF3240001616F7E0E20
:10243A00F4200001626F060E0001636F33EC16F0A0
:10244A0012000001E151040D1A0EF3240001616F1C
:10245A007F0EF4200001626F040E0001636F33ECFB
:10246A0016F012000001EC51060DD20EF324000101
:10247A00616F7E0EF4200001626F060E0001636F29
:10248A0033EC16F012000001F251050DF50EF3249B
:10249A000001616F7D0EF4200001626F050E0001DC
:1024AA00636F33EC16F012000001F551040DC30EF0
:1024BA00F3240001616F7F0EF4200001626F040EA5
:1024CA000001636F33EC16F01200000E0001616F19
:1024DA00000E606FACEC11F00001E26F040E000117
:1024EA00E26504D0000E0001E26F00D01200280E4F
:1024FA000001D06F040E0001D16F000E0001D56FEC
:10250A00080ED46F020E0001D66F230E0001D76F9A
:10251A000001D38F1200010E0001606F030E00014B
:10252A00E219D8B408D0040E0001E219D8B403D0D5
:10253A00000E0001606F0001605100D0120000011E
:10254A00F0510001F15DD8A002D0000E0BD00001BD
:10255A00F151010D000EF324D96E020EF420DA6E49
:10256A00DF5000D01200698468986D82010E000164
:10257A00E46F000E126E750E116E000E136E000ED1
:10258A00146E000E166E000E156EBFEC17F01200D8
:10259A0001C007F002C008F009D007C0D9FF08C07F
:1025AA00DAFF03C0DFFF074A082A00D00506D8A0D1
:1025BA0006060528F2E10628D8A4EFD71200000182
:1025CA00E22B040E0001E26504D0000E0001E26F66
:1025DA0000D08CEC11F0000E0001616F000E606FEC
:1025EA00E2C062F082EC14F0E2EC11F01200000199
:1025FA00E72B040E0001E76504D0000E0001E76F27
:10260A0000D08CEC11F0000E0001616F030E606FB8
:10261A00E7C062F082EC14F0F3EC11F01200000152
:10262A00E92B030E0001E96504D0000E0001E96FF1
:10263A0000D08CEC11F0000E0001616F060E606F85
:10264A00E9C062F082EC14F004EC12F0120000010E
:10265A00ED2B050E0001ED6504D0000E0001ED6FB3
:10266A0000D08CEC11F0000E0001616F010E606F5A
:10267A00EDC062F082EC14F015EC12F012000001C9
:10268A00E12B060E0001E16504D0000E0001E16FA6
:10269A0000D08CEC11F0000E0001616F050E606F26
:1026AA00E1C062F082EC14F026EC12F01200000194
:1026BA00EC2B050E0001EC6504D0000E0001EC6F56
:1026CA0000D08CEC11F0000E0001616F040E606FF7
:1026DA00ECC062F082EC14F037EC12F01200000148
:1026EA00F22B070E0001F26504D0000E0001F26F12
:1026FA0000D08CEC11F0000E0001616F020E606FC9
:10270A00F2C062F082EC14F048EC12F01200000100
:10271A00F52B020E0001F56504D0000E0001F56FDD
:10272A0000D08CEC11F0000E0001616F080E606F92
:10273A00F5C062F082EC14F059EC12F012000001BC
:10274A00626FFE0EF66E170EF76E0900020EF55E48
:10275A000900000EF55AD8A005D00001625160ECBC
:10276A0016F005D000016251E5EC14F000D0120019
:10277A000001626FFE0EF66E170EF76E0900020E6A
:10278A00F55E0900000EF55AD8A005D00001625185
:10279A00E5EC14F005D00001625160EC16F000D0AF
:1027AA00120060C066F061C067F00AD066C0D9FF47
:1027BA0067C0DAFF62C0DFFF0001664B672B00D0FB
:1027CA0000016407D8A0650700016429EFE1000150
:1027DA006529D8A4EBD712000001E551D8A416D078
:1027EA00000E6D6E000E696E160E6F6E9F0E6B6E8A
:1027FA007B0E696ED08EA28AA08AF28E01D06D8677
:10280A006DA6FDD7010E0001E56F00D01200000190
:10281A00685100016A03F3CF6CF0F4CF6DF0000148
:10282A00685100016B03F35000016D2700016951E3
:10283A0000016A03F35000016D276CC068F06DC097
:10284A0069F000D01200000E0001E46F000E126E53
:10285A00740E116E000E136E000E146E000E166EBC
:10286A00000E156EBFEC17F06D92699468B869A8EE
:10287A0004D0689802D0689400D068B4FCD71200DB
:10288A000001605100016111D8A402D0270E14D0B2
:10289A000001605100016111D8B40CD000016151EE
:1028AA0009E10A0E0001605DD8B004D00001605150
:1028BA001D0F02D02C0E00D012000C6E09A406D0F7
:1028CA00000E016E0C508AEC19F000D009A206D055
:1028DA00010E016E0C508AEC19F000D00C50010D5B
:1028EA00700EF3240A6E0F0EF4200B6E0AC0D9FF85
:1028FA000BC0DAFF09C0DFFF1200000E0001636F90
:10290A0060C0A9FF62C0A8FFA69EA69CA684000E6E
:10291A00F2BE010E0001636FF29E550EA76EAA0E5B
:10292A00A76EA68200D0A6B2FED7000163B102D07C
:10293A00F29E01D0F28EA69412006DA218D0010E5A
:10294A00A4EC13F0020EA4EC13F0030EA4EC13F0A3
:10295A0014D00DD00BEC16F010D0010EBDEC13F014
:10296A00020EBDEC13F0030EBDEC13F006D000010D
:10297A00E551200AD8B4EED7F0D7120070A01ED0C5
:10298A003BC0D9FF3CC0DAFF800EDE18D8A415D0B0
:10299A00D8C0D9FFD9C0DAFF840EDE18D8A40DD06A
:1029AA003BC0D9FF3CC0DAFF0C0EDF6E3BC0D9FF3B
:1029BA003CC0DAFF000EDB8E00D07090689A1200DD
:1029CA000001606F13D08CC1D9FF8DC1DAFF5A5054
:1029DA000BD08EC1D9FF8FC1DAFF5B5005D090C1F1
:1029EA00D9FF91C1DAFF5C50DF120CD000016051AF
:1029FA00010AD8B4E8D7030AD8B4EBD7010AD8B485
:102A0A00EED700D012000001E351D8B41ED0000165
:102A1A00E451D8B41AD0A09A0EEC0CF06D92180EAC
:102A2A0000016A6F5F0EE82EFED76A2FFCD700F00E
:102A3A006D84100E00016A6F940EE82EFED76A2F7D
:102A4A00FCD700D06D94A08A00D012000001F0518A
:102A5A000001F15DD8A002D0000E1CD00001F15196
:102A6A00010D000EF324D96E020EF420DA6EDF5047
:102A7A000001606F0001F12B000160510001D8A430
:102A8A0006D0000E0001F16F000E0001F06F000188
:102A9A00605100D012000001606F840E0001F161E4
:102AAA000ED00001F151010D000EF324D96E020E71
:102ABA00F420DA6E60C0DFFF0001F12B00D0840E33
:102ACA000001F1610CD00001F151010D000EF32457
:102ADA00D96E020EF420DA6E000EDF6E00D01200FC
:102AEA00000E0001656F06D00001665150EC15F02A
:102AFA000001652B00016551010D61C063F062C0E0
:102B0A0064F0F35000016327F4500001642363C0AA
:102B1A00F6FF64C0F7FF0800F5CF66F000D00001A9
:102B2A0066510001D8A4E0D71200FE0EF66E170E09
:102B3A00F76E0900030EF55E0900000EF55AD8A0DB
:102B4A000FD08B0E01018E6F0F0E01018F6F8EC198
:102B5A008CF18FC18DF1010E5A6E020E5B6E00D0A0
:102B6A00010EBDEC13F0020EBDEC13F0030EBDEC2A
:102B7A0013F012000001636F63C0EBF000016351B0
:102B8A0031EC1EF00001636FFE0EF66E170EF76E43
:102B9A000900030EF55E0900000EF55AD8B00CD0F4
:102BAA00512A5150800A7C0FD8A003D0000E516ED2
:102BBA0003D00001639300D00001635100D01200DA
:102BCA00000E38EC1CF09AEC15F096EC28F0F1ECBB
:102BDA0013F000D0A2EC14F0200E0001E56101D040
:102BEA00F9D76DA208D06FEC18F00009D8B4F2D763
:102BFA0008EC15F0EFD70001E451D8A4EBD701D0C7
:102C0A00E9D72EEC32F0E6D70CEF0CF005010851AB
:102C1A00BFEC15F00001646F000164A104D0010E3D
:102C2A00BDEC13F004D0010EA4EC13F000D00001A7
:102C3A0064A304D0020EBDEC13F004D0020EA4EC7F
:102C4A0013F000D0000164A504D0030EBDEC13F00C
:102C5A0004D0030EA4EC13F000D01200000E000101
:102C6A00676F06D00001665150EC15F00001672B22
:102C7A0000016751010D61C064F062C065F0F35054
:102C8A0000016427F4500001652364C0F6FF65C0A3
:102C9A00F7FF0800F5CF66F000D00001635100018C
:102CAA00675DD8B007D0000166510001D8B402D0E0
:102CBA00D9D700D012000001616F1ED05A50FF0A06
:102CCA000001606F8CC1D9FF8DC1DAFF11D05B5052
:102CDA00FF0A0001606F8EC1D9FF8FC1DAFF08D0E9
:102CEA005C50FF0A0001606F90C1D9FF91C1DAFF01
:102CFA0000016051DF160CD000016151010AD8B4FD
:102D0A00DDD7030AD8B4E3D7010AD8B4E9D700D08B
:102D1A001200020E4918D8A403D0B2EC26F027D02C
:102D2A00000E496E4150D8A41FD020EE01F03D504C
:102D3A00D9263E50DA22080EDF6E20EE02F03D5010
:102D4A00D9263E50DA22200EDE6E040EDD6E3DC01C
:102D5A00D9FF3EC0DAFF0C0EDF6E3DC0D9FF3EC080
:102D6A00DAFF000EDB8E03D0000E416E00D0120097
:102D7A00000E026E010E016EA2EC11F00001ED6F61
:102D8A00050E0001ED6504D0000E0001ED6F00D0C4
:102D9A00000E026E050E016EA2EC11F00001E16F49
:102DAA00060E0001E16504D0040E0001E16F00D0B7
:102DBA00000E026E060E016EA2EC11F00001E96F20
:102DCA00030E0001E96504D0000E0001E96F00D08E
:102DDA00120070C076F071C077F06EC074F06FC0E8
:102DEA0075F01CD076C0F6FF77C0F7FFF86A74C09A
:102DFA00D9FF75C0DAFF070EF76403D00800F55053
:102E0A0005D0F6CFE9FFF7CFEAFFEF50DF6E0001FA
:102E1A00764B772B0001744B752B00D0000172079B
:102E2A00D8A0730700017229DDE100017329D8A433
:102E3A00D9D71200000E0001616F010E606FACEC71
:102E4A0011F00001ED6F050E0001ED6504D0000ED2
:102E5A000001ED6F00D0000E0001616F050E606F7A
:102E6A00ACEC11F00001E16F060E0001E16504D03F
:102E7A00040E0001E16F00D0000E0001616F060E22
:102E8A00606FACEC11F00001E96F030E0001E96517
:102E9A0004D0000E0001E96F00D012000600EACF4C
:102EAA0026F0E1CF27F0E2CF28F0D9CF29F0DACF08
:102EBA002AF0F3CF2BF0F4CF2CF0F6CF2DF0F7CF8A
:102ECA002EF0F8CF2FF0F5CF30F0F1EC27F030C02C
:102EDA00F5FF2FC0F8FF2EC0F7FF2DC0F6FF2CC05C
:102EEA00F4FF2BC0F3FF2AC0DAFF29C0D9FF28C09C
:102EFA00E2FF27C0E1FF26C0EAFF25C0E9FF24C0A0
:102F0A00FBFF23C0FAFF110060C066F061C067F0E2
:102F1A001ED066C0F6FF67C0F7FFF86A070EF764AF
:102F2A0003D00800F55005D0F6CFE9FFF7CFEAFF46
:102F3A00EF5000016219D8A406D066C060F067C0DD
:102F4A0061F017D004D00001664B672B00D0000156
:102F5A006407D8A0650700016429DBE1000165293F
:102F6A00D8A4D7D7000E0001606F000E0001616F70
:102F7A0000D012000DD035D084EC11F032D088EC9C
:102F8A0011F02FD0BCEC2AF02CD043EC29F029D038
:102F9A0011C017F012C018F01850000AD8B404D0A3
:102FAA007F0AD8B41BD01DD01750010AD8B4EAD76B
:102FBA00030AD8B416D0010AD8B4E7D7060AD8B497
:102FCA0010D0770AD8B40DD0010AD8B40AD0070AAB
:102FDA00D8B4D5D7010AD8B4CFD703D01750FF0A2F
:102FEA0000D01200000E0001636F0001EA51D8B44C
:102FFA002FD060C0D9FF61C0DAFFDF500001626FD5
:10300A00DD0E00016217D8A423D0000120EE01F0E2
:10301A006051D9266151DA22DF500001626F050E34
:10302A0000016217D8A414D00001ED51D8B410D011
:10303A004A50D8B40AD0040E0001F219D8B408D004
:10304A00050E0001F219D8B403D0010E0001636F16
:10305A000001635100D0120000016B6F28D0010EED
:10306A000001EA6F33D0000E0001EA6F000E000182
:10307A00F46F2CD0000169510001D8B427D090EC2C
:10308A0012F00009D8B422D0010E4A1A1FD068C023
:10309A006AF0220E00016A17D8B418D090EC12F028
:1030AA000009D8B413D0870E00016B6F0FD000014E
:1030BA006B51270AD8B4EBD71E0AD8B4DBD7A90AB2
:1030CA00D8B4CDD7010AD8B4CED700D000016B51FD
:1030DA0000D01200FE0EF66E170EF76E0900030EF0
:1030EA00F55E0900000EF55AD8A006D0010E0001BF
:1030FA00F66F070E5E6E00D0FE0EF66E170EF76EB6
:10310A000900040EF55E0900000EF55AD8A003D096
:10311A00F30E5D6E00D0F6C092FF000E966E010EA1
:10312A000001626F8350FF0A5D140009D8A40DD014
:10313A008150FF0A0001606F3F0E00016017D8A49A
:10314A0004D0000E0001626F00D062C061F03F0E31
:10315A00926E5EC096FF0001615100D0120033D01A
:10316A0062C0D9FF63C0DAFF60C0E1FF61C0E2FF5D
:10317A00DE50E618D8B420D062C0D9FF63C0DAFFA7
:10318A00DF500001666F676B0001661F671F664BA1
:10319A00672B60C0D9FF61C0DAFFDF500001686F9A
:1031AA0000016851000166250001606F000E0001F0
:1031BA0067210001616F18D00001604B612B00018B
:1031CA00624B632B00D000016407D8A06507000199
:1031DA006429C6E100016529D8A4C2D7000E0001FE
:1031EA00616F000E606F00D01200000E4D6E000E6F
:1031FA00446E000E426E000E436E000E416E000ECB
:10320A00496ED8C0D9FFD9C0DAFF7F0EDF16040E87
:10321A000001D81BD8C0D9FFD9C0DAFF7F0EDF164C
:10322A00040E0001D81B3DC0D9FF3EC0DAFF7F0E55
:10323A00DF16000E0001FA6F000E0001FC6F000E8F
:10324A00FB6F000E0001D36F000E0001D56F000E58
:10325A00D46F48EC21F0000E126E030E116E000EB0
:10326A00136E000E146E000E166E000E156EBFEC75
:10327A0017F03AEC22F01200830F830F830F830FAB
:10328A00830F830F810F810F810F810F810F810FB0
:10329A00810F810F810F810F810F810F830F830FA0
:1032AA00830F830F830F830F920F920F920F920F48
:1032BA00920F920F960F960F960F960F960F920FE8
:1032CA00920F920F920F920F102040800408201044
:1032DA00020104088040201008042010080401029A
:1032EA000102040810208040201002010102040893
:1032FA001020010202040810200102040402012025
:10330A00100804028C0F8C0F8B0F066E000E076ECE
:10331A00040E086E0150026E036AD8900236033614
:10332A000650046E056AD89004360536D8900436DD
:10333A0005360250042603500522D8900436053675
:10334A00D89004360536045007260550082207C0CF
:10335A00D9FF08C0DAFFDF9E0150D8A407D0065073
:10336A00020D370EF324D96E000E06D00650020D58
:10337A00D80EF324D96E000EF420DA6E07C0DEFFF1
:10338A0008C0DDFF00D007C0D9FF08C0DAFFDF9C04
:10339A0020EE04F00750D9260850DA22DF8C1200FA
:1033AA0002EE00F0840EEE6AE806FDE101EE92F00C
:1033BA00580EEE6AE806FDE100EED0F02D0EEE6A38
:1033CA00E806FDE100EE31F0290EEE6AE806FDE1BD
:1033DA00820EF66E320EF76E000EF86E01EE00F0F7
:1033EA0010EE92F00900F5CFEEFFE550E150FAE158
:1033FA00FA0EF66E220EF76E000EF86E0900F5CF81
:10340A00FDF00900F5CFFEF00900F5CFFFF0FD0E43
:10341A00F66E220EF76E000EF86E00EE5AF010EEFF
:10342A0005F00900F5CFEEFFE550E150FAE1000E94
:10343A00F86E0001E5EF15F0000E426E000E436EC5
:10344A00020E4918D8A41DD020EE01F03D50D9260D
:10345A003E50DA22080EDF6E20EE02F03D50D926E9
:10346A003E50DA22280EDE6E040EDD6E3DC0D9FF14
:10347A003EC0DAFF480EDF6E3DC0D9FF3EC0DAFF1C
:10348A0026D00001FB510401265D0001FC51040114
:10349A002759D8B005D026C4FBF027C4FCF000D0C9
:1034AA005BEC20F0000120EE02F0D851D926D95168
:1034BA00DA22280EDE6E040EDD6ED8C0D9FFD9C01E
:1034CA00DAFF480EDF6ED8C0D9FFD9C0DAFF000E86
:1034DA00DB8E00D012000001706F70C060F0000136
:1034EA00616B000E0001636F0C0E626FC2EC1AF082
:1034FA00000160510001716F0001EBA13BD0060E83
:10350A000001716537D0070E0001715F000E0001DE
:10351A00636F0C0E626F70C060F00001616BC9ECE2
:10352A001DF060C068F061C069F0000E00016B6FA9
:10353A00050E6A6F0CEC14F0450E00016E6F770EE3
:10354A0000016F6F0001685100016E270001695187
:10355A0000016F2300017151010DF35000016E2724
:10356A00F45000016F236EC0F6FF6FC0F7FF08002A
:10357A00F55002D0000E00D01200000E0001656F57
:10358A00000161AF09D00001606D611FD8B0612BE5
:10359A00010E0001656F00D0000163AF06D0000183
:1035AA00626D631FD8B0632B00D000016251000125
:1035BA006311D8B42BD0010E0001646F07D000014B
:1035CA00D890623763370001642B00D0000163BFD3
:1035DA0002D0F5D700D0000162510001605D000100
:1035EA00635100016159D8A009D00001625100015C
:1035FA00605F000163510001615B00D00001D89057
:10360A00633362330001642FE6D700D000016551AD
:10361A000001D8B406D00001606D611FD8B0612BDB
:10362A0000D060C060F061C061F000D012000001FB
:10363A00726F780E0001706F7D0E0001716F000EBF
:10364A000001736F00017351800A790FD8B048D016
:10365A0001D046D0000173510001686F696B68BFE1
:10366A006907000E00016B6F010E6A6F0CEC14F013
:10367A0070C06EF071C06FF00001685100016E27D2
:10368A000001695100016F236EC0F6FF6FC0F7FF9A
:10369A000800F55000017219D8A41FD00001EC519E
:1036AA00070D780E00016E6F7D0E00016F6FF350EB
:1036BA0000016E27F45000016F2300017351010DC0
:1036CA00F35000016E27F45000016F236EC0F6FF1D
:1036DA006FC0F7FF0800F55006D00001732BB2D770
:1036EA000001725100D012000A6E51D0000EBD6E58
:1036FA00000EBA6E0F0EC16EFE0EF66E170EF76E44
:10370A000900030EF55E0900000EF55AD8A019D07B
:10371A00000EC26E0E0EC16E9E0EC06EFE0EF66ECC
:10372A00170EF76E0900030EF5180900F510D8A454
:10373A0002D0FE0E01D0F30E0001FE6F070E00014B
:10374A00FF6F000E896E3F0E926E000E8A6E9368AE
:10375A00F19E000E8B6E380E946E000E8C6EFEC0BB
:10376A0095FF848E000E8D6EFFC096FFB9EC22F095
:10377A0019D0130ED36E16D0600ED36E100E096ECA
:10378A00940EE82EFED7092EFCD700D00BD00A5093
:10379A00000AD8B4ABD7010AD8B4EBD7030AD8B415
:1037AA00EBD700D01200056E0150D8B407D00550EF
:1037BA00020DD80EF324D96E000E06D00550020D64
:1037CA00370EF324D96E000EF420DA6EDECF06F03F
:1037DA00DDCF07F000D006500710D8A405D0000EA0
:1037EA00016E000E026E3ED020EE02F00650D9267F
:1037FA000750DA2202C0DEFF03C0DDFF20EE01F02F
:10380A000650D9260750DA2204C0DFFF06C0D9FFC6
:10381A0007C0DAFF400EDF1606C0D9FF07C0DAFF7D
:10382A00000EDB8606C0D9FF07C0DAFF000EDB8E6A
:10383A000150D8B407D00550020DD80EF324D96E22
:10384A00000E06D00550020D370EF324D96E000E75
:10385A00F420DA6E040EDF1A00D006C001F007C0A9
:10386A0002F000D012000001696F52D0000EBD6E46
:10387A00000EBA6E0F0EC16EFE0EF66E170EF76EC2
:10388A000900030EF55E0900000EF55AD8A019D0FA
:10389A00000EC26E0E0EC16E9E0EC06EFE0EF66E4B
:1038AA00170EF76E0900030EF5180900F510D8A4D3
:1038BA0002D0FE0E01D0F30E0001FE6F070E0001CA
:1038CA00FF6F000E896E3F0E926E000E8A6E93682D
:1038DA00F19E000E8B6E380E946E000E8C6EFEC03A
:1038EA0095FF848E000E8D6EFFC096FF78EC25F052
:1038FA001BD0130ED36E18D0600ED36E100E0001BB
:10390A00686F940EE82EFED7682FFCD700D00CD033
:10391A0000016951000AD8B4A9D7010AD8B4E9D775
:10392A00030AD8B4E9D700D012004550D8A45FD012
:10393A00010E456E4650D8A45AD0010E466E020EAC
:10394A004918D8A416D0000120EE01F0D851D92682
:10395A00D951DA22000EDF6ED8C0D9FFD9C0DAFFFA
:10396A00480EDF6ED8C0D9FFD9C0DAFF000EDB8E51
:10397A003ED04904D8A43BD0000E416E20EE01F09F
:10398A003B50D9263C50DA22080EDF6E20EE02F0B8
:10399A003B50D9263C50DA22200EDE6E040EDD6E34
:1039AA003BC0D9FF3CC0DAFF040EDF6E3BC0D9FF33
:1039BA003CC0DAFF000EDB8E010E416E20EE01F0F4
:1039CA003D50D9263E50DA22080EDF6E20EE02F074
:1039DA003D50D9263E50DA22200EDE6E040EDD6EF0
:1039EA003DC0D9FF3EC0DAFF800EDF6E00D0120064
:1039FA00000E0401286F000E0401296F41D0000156
:103A0A00FA8F03D00401288100D00001E305D8A46D
:103A1A0043D00401288340D00001FA8F3DD0000131
:103A2A00FA8F040124BF0BD0040124510F0B016E3D
:103A3A000150020D370EF324D96E000E0AD004018C
:103A4A0024510F0B016E0150020DD80EF324D96ECA
:103A5A00000EF420DA6EDECF02F0DDCF03F000D0E4
:103A6A0002C0D9FF03C0DAFFDFAE16D002C0D9FF09
:103A7A0003C0DAFFDFA410D0010E0401286F0CD0B6
:103A8A00040120511F0B000AD8B4B9D7010AD8B4CF
:103A9A00C3D7030AD8B4C3D70001FAAF0CD0280E93
:103AAA000001F76F040E0001F86F0001FA81020E9F
:103ABA000001FB6F00D012002D0E476E57C01FF099
:103ACA00FD0E1F16D8A457D057C01FF0D8901F322A
:103ADA003F0E1F161F50040D000EF3243B6E040EFA
:103AEA00F4203C6E3BC03DF03CC03EF0040E3D1A53
:103AFA003BC0D9FF3CC0DAFFDF30E8320F0B0D0ABA
:103B0A00D8A436D0000E216E070E216401D023D02E
:103B1A0020EE02F03B50D9263C50DA22DECF1FF0CD
:103B2A00DDCF20F01FC0D9FF20C0DAFF2150010DE0
:103B3A00200EF324E16E040EF420E26EDFCFE7FFDD
:103B4A0020EE02F03B50D9263C50DA22DE2A000E43
:103B5A00DD22212AD9D720EE02F03B50D9263C504B
:103B6A00DA22200EDE6E040EDD6EFAEC18F00BD0AF
:103B7A008EEC16F008D05750FD0B040AD8A403D0D7
:103B8A009BEC1EF000D01200000E0001656F0001D0
:103B9A0063AF09D00001626D631FD8B0632B010EB9
:103BAA000001656F00D0000161AF09D00001606DAE
:103BBA00611FD8B0612B010E0001651B00D0000EF9
:103BCA000001676F000E666F000162510001631108
:103BDA00D8B431D0010E0001646F07D00001D8902B
:103BEA00623763370001642B00D0000163BF02D043
:103BFA00F5D700D00001D8906637673700016251C7
:103C0A000001605D0001635100016159D8A00BD029
:103C1A00000162510001605F000163510001615BB4
:103C2A000001668100D00001D8906333623300013D
:103C3A00642FE0D700D0000165510001D8B406D046
:103C4A000001666D671FD8B0672B00D066C060F0B0
:103C5A0067C061F000D012000001626F0001ED51EF
:103C6A00D8A43AD05FD038D000D0E1C060F0010EBD
:103C7A000001616F0001602B03D00001D890613709
:103C8A000001602FFAD700016151FF0A0001621793
:103C9A00E1C060F0EAC061F00001602B03D00001CE
:103CAA00D89061370001602FFAD711D000D0E1C057
:103CBA0060F0FD0E00016027EAC061F00001602B90
:103CCA0003D00001D89061370001602FFAD70001B4
:103CDA0061510001621315D00001E151000AD8B404
:103CEA00C4D7010AD8B4C1D7030AD8B4BED7010AC7
:103CFA00D8B4DDD7070AD8B4DAD7010AD8B4D7D7E7
:103D0A0000D0020E0001F519D8A40CD00001F4A3CA
:103D1A0003D00001628100D00001F4AB03D000019E
:103D2A00628500D00001625100D01200D8C0D9FFCC
:103D3A00D9C0DAFF000EDFBC010E026E040E0001CC
:103D4A00D81B080E0001E519D8A40DD00401225190
:103D5A007F0B6E6E6E50D8B402D0100E01D0040ED6
:103D6A000001E56F00D04904D8A430D0000120EE4C
:103D7A0002F0D851D926D951DA22280EDE6E040E65
:103D8A00DD6E5BEC20F0020E4D18D8A40DD0D8C021
:103D9A00D9FFD9C0DAFF040E16D0D8C0D9FFD9C0CE
:103DAA00DAFF000EDB8E2FD00250D8A407D0D8C07D
:103DBA00D9FFD9C0DAFF480E06D0EFD7D8C0D9FF4D
:103DCA00D9C0DAFF080EDF6EE8D71DD00001D3AFE5
:103DDA0017D00001D6510001D711D8B40ED020EE69
:103DEA00D6F001D80AD00500FA6EDE50FD6EDE501C
:103DFA00FE6EF850FF6EFA5012000001D39F00D0F9
:103E0A00000E496E00D012000001646F000160517B
:103E1A000001D8B408D000016451020DD80EF32471
:103E2A00D96E000E07D000016451020D370EF3243B
:103E3A00D96E000EF420DA6EDECF65F0DDCF66F0C3
:103E4A0000D00001655100016611D8A407D0000E08
:103E5A000001606F000E0001616F44D0000120EE86
:103E6A0002F06551D9266651DA2261C0DEFF62C0CE
:103E7A00DDFF000120EE01F06551D9266651DA22F4
:103E8A0063C0DFFF65C0D9FF66C0DAFF400EDF16E8
:103E9A0065C0D9FF66C0DAFF000EDB8665C0D9FFB0
:103EAA0066C0DAFF000EDB8E000160510001D8B453
:103EBA0008D000016451020DD80EF324D96E000E09
:103ECA0007D000016451020D370EF324D96E000E9B
:103EDA00F420DA6E040EDF1A00D065C060F066C006
:103EEA0061F000D01200000E00016A6F000E00019E
:103EFA006B6F000E00016D6F070E00016D6501D03A
:103F0A0011D000016D51010DDF0EF324D96E010E9F
:103F1A00F420DA6E010EDF6402D000016A2B000180
:103F2A006D2BEAD7000E00016D6F0B0E00016D6557
:103F3A0001D011D000016D51010DC30EF324D96EC9
:103F4A00010EF420DA6E010EDF6402D000016B2B41
:103F5A0000016D2BEAD7000E00016C6F010E000103
:103F6A006A6508D0010E00016B6504D0010E0001DC
:103F7A006C6F00D06CC069F0DF0E0001606F010E3B
:103F8A000001616F000E0001636F000E626F000E88
:103F9A000001656F080E646FD6EC13F0C30E0001C2
:103FAA00606F010E0001616F000E0001636F000E69
:103FBA00626F000E0001656F0C0E646FD6EC13F091
:103FCA000001695100D012000001FA8F710E016ED2
:103FDA000F0E026E000E046E000E036E000E066EC9
:103FEA00010E056ECDEC12F0000E016E040E026E8B
:103FFA00000E046E000E036E000E066E200E056E95
:10400A00CDEC12F06D8C000E196E010E196401D000
:10401A0016D01950010DDC0EF324D96E000EF420CF
:10402A00DA6E000EDF6E1950010DDE0EF324D96E22
:10403A00000EF420DA6E000EDF6E192AE6D7560E4D
:10404A00016E000E026E000E046E000E036E000E6C
:10405A00066E010E056ECDEC12F06D9C080E000185
:10406A00D86F040E0001D96F000E3B6E040E3C6E31
:10407A003BC03DF03CC03EF022C455F05550D8A498
:10408A0002D0100E0FD0000E126E010E116E550ED8
:10409A00136E000E146E000E166E010E156EBFEC36
:1040AA0017F0200E0001E56F00D01200080E016E15
:1040BA000001FC5112E1080E0001FB5DD8B00DD0E1
:1040CA00FBC001F04D50D8A402D0010E04D04D041B
:1040DA00D8A403D0020E4D6E00D001500001FB5F40
:1040EA00000EFC5B000120EE01F0D851D926D9510F
:1040FA00DA2201C0DFFF280E01019B6F040E0101C5
:10410A009C6F0001FAA11FD041D01DD0F7C0F6FF65
:10411A00F8C0F7FFF86A9BC1D9FF9CC1DAFF070E06
:10412A00F76403D00800F55005D0F6CFE9FFF7CFC2
:10413A00EAFFEF50DF6E0001F74BF82B01019B4BB2
:10414A009C2B010600D00150D8B425D0DFD723D04C
:10415A001DD0F7C0F6FFF8C0F7FFF86A9BC1D9FF78
:10416A009CC1DAFF070EF76403D00800F55005D0AA
:10417A00F6CFE9FFF7CFEAFFEF50DF6E0001F74B0A
:10418A00F82B01019B4B9C2B010600D00150D8B49F
:10419A0002D0DFD700D012000001726F040E0001B6
:1041AA00F219D8B405D0050E0001F219D8A423D00B
:1041BA004F0E000172651FD0540E000172611BD0B0
:1041CA00B00E000172250001686F0001696BFF0ED5
:1041DA006923000E00016B6F030E6A6F0CEC14F07A
:1041EA00B70E0001682500016E6F7F0E000169217C
:1041FA0046D048D000D0000E0001636F0C0E626FEB
:10420A0072C060F00001616BC9EC1DF060C068F01B
:10421A0061C069F0000E00016B6F240E6A6F0CEC2E
:10422A0014F0840E0001706F770E0001716F0001A7
:10423A006851000170270001695100017123000EC5
:10424A000001636F0C0E626F72C060F00001616B57
:10425A00C2EC1AF060C068F061C069F0000E00019B
:10426A006B6F030E6A6F0CEC14F0000168510001C9
:10427A00702500016E6F0001695100017121000172
:10428A006F6F00D0120004012039E832030B0009D5
:10429A00D8A470D04DD06ED04BD00001FA8F080E42
:1042AA000001E56F67D051EC27F064D0E9EC1FF00C
:1042BA0061D0550E0001F76F000E16D00001FA8189
:1042CA0016D00001FA8F56D0FDEC1CF053D000D066
:1042DA00A4EC2BF04FD004012451010D560EF32407
:1042EA000001F76F000EF4200001F86FE7D7010E06
:1042FA000001FB6FE6D70001FA8F04012451010D7A
:10430A00560EF324D96E000EF420DA6E22C4DFFFB3
:10431A0031D0000E126E020E116E000E136E000ED8
:10432A00146E000E166E000E156EBFEC17F022D03A
:10433A0004012151000AD8B4C7D7010AD8B4C8D792
:10434A00020AD8B4C5D7060AD8B4A7D7030AD8B47C
:10435A00AAD7010AD8B4DDD70F0AD8B4AAD7010A56
:10436A00D8B4A4D7030AD8B4B6D7010AD8B4C3D7E5
:10437A00070A00D0120070C078F071C079F06EC0E0
:10438A0076F06FC077F0000176510001785D000188
:10439A00775100017959D8B045D000017251000116
:1043AA0078250001746F0001735100017921000121
:1043BA00756F000174510001765D000175510001AD
:1043CA007759D8B02FD00001725100017827000127
:1043DA00735100017923000172510001762700010F
:1043EA0073510001772300D000017807D8A079071C
:1043FA0078C0D9FF79C0DAFF00017607D8A077071D
:10440A0076C0E1FF77C0E2FFDFCFE7FF0001720766
:10441A00D8A073070001725100017311D8B424D0D7
:10442A00E3D722D00001725100017311D8B41CD015
:10443A0078C0D9FF79C0DAFF76C0E1FF77C0E2FF22
:10444A00DFCFE7FF0001784B792B0001764B772B02
:10445A0000017207D8A0730700017251000173119D
:10446A00D8B402D0E5D700D012006D980001FABF87
:10447A003BD00001D3AF0DD0020E496E4350D8A4F1
:10448A0003D021EC1AF000D0000E466E000E456EE5
:10449A006AD020EE01F03D50D9263E50DA22080EAD
:1044AA00DF6E20EE02F03D50D9263E50DA22200E71
:1044BA00DE6E040EDD6E3DC0D9FF3EC0DAFF0C0E83
:1044CA00DF6E3DC0D9FF3EC0DAFF000EDB8ED8C0DA
:1044DA00D9FFD9C0DAFF040EDF6ED8C0D9FFD9C020
:1044EA00DAFF000EDB8E3FD0040120AF12D0010E9E
:1044FA00496E4250D8A403D021EC1AF000D0000E25
:10450A00466E000E456E4450D8A42DD09AEC1CF08D
:10451A002AD0020E496E20EE01F03D50D9263E50B7
:10452A00DA22080EDF6E20EE02F03D50D9263E5008
:10453A00DA22200EDE6E040EDD6E3DC0D9FF3EC0CB
:10454A00DAFF040EDF6E3DC0D9FF3EC0DAFF000E6F
:10455A00DB8E000E466E000E456E4450D8A403D082
:10456A009AEC1CF000D012009F0E016E010E026E32
:10457A00000E046E0E0E036E000E066E240E056EFD
:10458A00CDEC12F0000E0001E86FCF0E016E010EA5
:10459A00026E000E046E000E036E000E066E080E0A
:1045AA00056ECDEC12F0D70E016E010E026E000EF2
:1045BA00046E000E036E000E066E020E056ECDEC42
:1045CA0012F0D90E016E010E026E000E046E0E0E6E
:1045DA00036E000E066E060E056ECDEC12F0000E8E
:1045EA000001EF6FEFC0EEF0020E0001E66F000E61
:1045FA00026E020E016EA2EC11F00001F26F070EBC
:10460A000001F26504D0000E0001F26F00D0000E26
:10461A00026E040E016EA2EC11F00001EC6F050EA1
:10462A000001EC6504D0000E0001EC6F00D0000E12
:10463A00026E030E016EA2EC11F00001E76F040E88
:10464A000001E76504D0000E0001E76F00D0000EFC
:10465A00026E080E016EA2EC11F00001F56F020E57
:10466A000001F56504D0000E0001F56F00D0D1EC11
:10467A0011F0BDEC16F012000001766F00017651C0
:10468A0070EC1AF00001776F76C060F00001616B80
:10469A00000E0001636F0C0E626FC9EC1DF0000181
:1046AA0060510001786F76C060F00001616B000E06
:1046BA000001636F0C0E626FC2EC1AF000016051C8
:1046CA000001796F000177510001D8B445D000018B
:1046DA00775159D041D020D0000178510C0DC50E28
:1046EA000001746F750E1FD0000178510C0D650E14
:1046FA000001746F750E17D0000178510C0D250E4C
:10470A000001746F760E0FD0000178510C0D850EE2
:10471A000001746F760E07D0000178510C0DE50E7A
:10472A000001746F760E0001756FF3500001742753
:10473A00F4500001752300017951010DF350000175
:10474A007427F4500001752374C0F6FF75C0F7FF93
:10475A000800F5CF77F012D00001E251000AD8B470
:10476A00DBD7010AD8B4B8D7030AD8B4BDD7010A2F
:10477A00D8B4C2D7070AD8B4C7D7CED70001775161
:10478A001CEC1BF000D0120000017E6FFE0EF66ECC
:10479A00170EF76E0900020EF55E0900000EF55AB3
:1047AA00D8A020D000017E510C0D050E00017B6FB0
:1047BA00750E00017C6FF35000017B27F450000155
:1047CA007C2300017A51010DF35000017B27F4503C
:1047DA0000017C237BC0F6FF7CC0F7FF0800F5CF01
:1047EA007DF009D000017E510C0DF35000017A25AD
:1047FA0000017D6F00D000017A51010DC30EF32430
:10480A00D96E010EF420DA6EDF2A00017E51010D05
:10481A00DF0EF324D96E010EF420DA6EDF2A0001CE
:10482A007D5141EC23F000017F6FDF0E00017F65AF
:10483A001AD0E80E00017F6116D07FC07BF0200EEF
:10484A0000017B27010E00017C6F00017B2B03D046
:10485A000001D8907C3700017B2FFAD700017C51E8
:10486A000001EE131CD0F00E00017F19D8A403D06A
:10487A000101D08114D00001E651800A780FD8B026
:10488A000ED00001E651010DCF0EF324D96E010EB0
:10489A00F420DA6E7DC0DFFF0001E62B00D01200A3
:1048AA007AC0D9FF7BC0DAFFDF500001816F0001B7
:1048BA0020EE01F07A51D9267B51DA220001DFB4C9
:1048CA0076D0020E0001806F020E0001836F000194
:1048DA008351800A780FD8B06AD001D068D000011D
:1048EA0083510001686F696B68BF6907000E000198
:1048FA006B6F010E6A6F0CEC14F000016851000135
:10490A007A25D96E0001695100017B21DA6EDF50E8
:10491A000001826F0001825170EC1AF00001846F6D
:10492A00000184510001D8A407D00001825141EC52
:10493A0023F00001846F00D081C068F0020E0001EC
:10494A007C250001606F000E00017D210001616F6E
:10495A0084C062F00001636B000E0001656F060EF1
:10496A00646F89EC17F00001605100016111D8A44D
:10497A0002D0010E01D0000E0001696F00018451BE
:10498A0031EC18F00001846F00018051010DF350E1
:10499A0000017E25D96EF45000017F21DA6E84C0B1
:1049AA00DFFF0001802B0001832B91D700D07EC04E
:1049BA00D9FF7FC0DAFF81C0DFFF010E00D01200ED
:1049CA00690E0001616F7F0E0001626F75EC15F0D0
:1049DA00FE0EF66E170EF76E0900F5CF60F00A00AC
:1049EA00F5CF61F045EC14F050EC15F0280E50ECC0
:1049FA0015F0CF0E0001616F7F0E0001626F75EC3A
:104A0A0015F0000E0001616F000E606F45EC14F0A6
:104A1A0050EC15F0370E50EC15F0000E0001616FE6
:104A2A00010E606F45EC14F050EC15F0000E000119
:104A3A00616F070E606F45EC14F050EC15F0280E0C
:104A4A0050EC15F01D0E0001616F7E0E0001626FC1
:104A5A0075EC15F048EC12F0DE0E0001616F7F0E66
:104A6A000001626F75EC15F0E2EC11F0E20E000144
:104A7A00616F7F0E0001626F75EC15F015EC12F094
:104A8A00E60E0001616F7F0E0001626F75EC15F092
:104A9A00F3EC11F0EA0E0001616F7F0E0001626F04
:104AAA0075EC15F037EC12F0EE0E0001616F7F0E17
:104ABA000001626F75EC15F004EC12F0F20E0001C1
:104ACA00616F7F0E0001626F75EC15F026EC12F033
:104ADA00DA0E0001616F7F0E0001626F75EC15F04E
:104AEA0059EC12F012009F0E0001606F010E0001D6
:104AFA00616F000E0001636F0E0E626F000E0001FF
:104B0A00656F240E646FD6EC13F0000E0001E86F97
:104B1A00CF0E0001606F010E0001616F000E0001EF
:104B2A00636F000E626F000E0001656F080E646FFE
:104B3A00D6EC13F0D70E0001606F010E0001616F11
:104B4A00000E0001636F000E626F000E0001656FB8
:104B5A00020E646FD6EC13F0D90E0001606F010EDD
:104B6A000001616F000E0001636F0E0E626F000E8E
:104B7A000001656F060E646FD6EC13F0000E00019B
:104B8A00EF6FEFC0EEF0020E0001E66F000E0001BB
:104B9A00616F020E606FACEC11F00001F26F070E4C
:104BAA000001F26504D0000E0001F26F00D0000E81
:104BBA000001616F040E606FACEC11F00001EC6F44
:104BCA00050E0001EC6504D0000E0001EC6F00D068
:104BDA00000E0001616F030E606FACEC11F0000172
:104BEA00E76F040E0001E76504D0000E0001E76FCD
:104BFA0000D0000E0001616F080E606FACEC11F07E
:104C0A000001F56F020E0001F56504D0000E0001E7
:104C1A00F56F00D06AEC12F01FEC17F01200A09AA0
:104C2A00000E6A6E000E686E000E706E710E016ED6
:104C3A000F0E026E000E046E000E036E000E066E5C
:104C4A00010E056ECDEC12F0160E6F6E9F0E6B6E96
:104C5A007B0E696E000E096E0ED010D00950040D3D
:104C6A00000EF324D96E040EF420DA6EDE6ADE6AD0
:104C7A00DE6ADD6A092A070E0964F0D76D8C000E18
:104C8A006E6E6D986D9C0DD06896000E0001FA6FDD
:104C9A00000E0001D36F000E0001D56F000ED46F15
:104CAA0000D068B6F1D7010E456E010E466E000EB1
:104CBA00426E000E436E000E0001E46F000E096E94
:104CCA00010E096401D02ED00950020DD80EF3242A
:104CDA00D96E000EF420DA6E000EDE6E000EDD6E66
:104CEA000950020D370EF324D96E000EF420DA6E45
:104CFA00000EDE6E000EDD6E0950010DDC0EF3248F
:104D0A00D96E000EF420DA6E000EDF6E0950010D26
:104D1A00DE0EF324D96E000EF420DA6E000EDF6E7A
:104D2A00092ACED7080E0001D86F040E0001D96FE8
:104D3A00160E706E040E0401036F200E026F080E29
:104D4A000401016F040E0401006F0401008F000EBC
:104D5A00556E000E0001E56F120020EE01F03B5087
:104D6A00D9263C50DA22DF50026E02500001D45D8F
:104D7A00000ED559D8B003D0D4C002F000D00250EA
:104D8A000001D45F000ED55B000E016E13D00150F6
:104D9A00010D280EF324D96E040EF420DA6ED0C069
:104DAA00E1FFD1C0E2FFDFCFE7FF0001D04BD12BFB
:104DBA00012A00D00250015CD8A0E9D70001D451E1
:104DCA000001D511D8B42DD020EE01F03D50D926DE
:104DDA003E50DA22080EDF6E20EE02F03D50D92650
:104DEA003E50DA22280EDE6E040EDD6E3BC0D9FF7D
:104DFA003CC0DAFFDFBC0DD03DC0D9FF3EC0DAFFB0
:104E0A00480E0CD03DC0D9FF3EC0DAFF000EDB8E43
:104E1A0042D03DC0D9FF3EC0DAFF080EDF6EF2D79E
:104E2A003AD020EE01F03D50D9263E50DA22080E43
:104E3A00DF6E20EE02F03D50D9263E50DA22200ED7
:104E4A00DE6E040EDD6E3DC0D9FF3EC0DAFF040EF1
:104E5A00DF6E3DC0D9FF3EC0DAFF000EDB8E0001D7
:104E6A00D6510001D711D8B40ED020EED6F001D811
:104E7A000AD00500FA6EDE50FD6EDE50FE6EF85066
:104E8A00FF6EFA5012000001D39F4450D8A403D0F9
:104E9A009AEC1CF000D01200800E04012019D8A44C
:104EAA009AD0C00E0001FA6F89D0A50E0001F76FE3
:104EBA007F0E0001F86F000E0001FC6F120EFB6FEF
:104ECA008AD004012251D8A444D004012251020DEF
:104EDA00820EF324F66E770EF420F76E0900F5CFF2
:104EEA00F7F00A00F5CFF8F0020E0001F725016E7F
:104EFA00000E0001F821026E01C0F6FF02C0F7FFA2
:104F0A00F86A070EF76403D00800F55005D0F6CF0B
:104F1A00E9FFF7CFEAFFEF500001FB6F030E000134
:104F2A00F725016E000E0001F821026E01C0F6FF9E
:104F3A0002C0F7FFF86A070EF76403D00800F550BD
:104F4A0005D0F6CFE9FFF7CFEAFFEF500001FC6F7B
:104F5A0042D0000E0001FA6F3ED0030E0401226116
:104F6A0025D004012251020D740EF324F66E770E39
:104F7A00F420F76E0900F5CFF7F00A00F5CFF8F044
:104F8A00F7C0F6FFF8C0F7FFF86A070EF76403D018
:104F9A000800F55005D0F6CFE9FFF7CFEAFFEF504A
:104FAA00016E01500001FB6FFC6B15D0000E000171
:104FBA00FA6F11D0000E0001FA6F0DD004012351CF
:104FCA00010AD8B472D7030AD8B47BD7010AD8B475
:104FDA00C4D7F0D700D012000001E505D8B46DBAE5
:104FEA0008D0000E686E69806988020E0001E56FBC
:104FFA0000D068B469A404D0689428EC14F000D0F6
:10500A006DB28DD068B069A008D014EC26F0A08AE1
:10501A00040E0001E56F689000D068B869A804D052
:10502A00B8EC12F0689800D068AC1DD069AC0FD00B
:10503A00000E126E730E116E000E136E000E146EB9
:10504A00000E166E010E156EBFEC17F000D0689CAC
:10505A004750D8B402D0470600D04750D8A403D04E
:10506A009AEC1CF000D068BA69AA03D0C3EC14F019
:10507A0000D068B269A210D07F0E126E1168000EBD
:10508A00136E000E146E000E166E010E156EBFEC36
:10509A0017F0000E6A6E00D0040E0001E56101D01F
:1050AA003ED069A63CD0000E226E030E226401D0C7
:1050BA0036D068A634D06CCF57F05730E832E83291
:1050CA000F0B4B6E689657B407D04B50010DDE0E8E
:1050DA00F324D96E000E06D04B50010DDC0EF324DA
:1050EA00D96E000EF420DA6E0001DF7000D04B504A
:1050FA00D8A403D061EC1DF010D0000E126E720E0F
:10510A00116E570E136E000E146E000E166E000E00
:10511A00156EBFEC17F001D002D0222AC6D7A19A89
:10512A001200A09A000E6A6E000E686E000E706E73
:10513A00710E0001606F0F0E0001616F000E000119
:10514A00636F000E626F000E0001656F010E646FDF
:10515A00D6EC13F0160E6F6E9F0E6B6E7B0E696E99
:10516A00000E0001686F10D013D000016851040DC1
:10517A00000EF324D96E040EF420DA6EDE6ADE6ABB
:10518A00DE6ADD6A0001682B070E00016865EDD74B
:10519A006D8C000E6E6E6D986D9C0DD06896000E2B
:1051AA000001FA6F000E0001D36F000E0001D56FE7
:1051BA00000ED46F00D068B6F1D7010E456E010E0D
:1051CA00466E000E426E000E436E000E0001E46F42
:1051DA00000E0001686F010E0001686501D033D02E
:1051EA0000016851020DD80EF324D96E000EF42086
:1051FA00DA6E000EDE6E000EDD6E00016851020DE1
:10520A00370EF324D96E000EF420DA6E000EDE6E2D
:10521A00000EDD6E00016851010DDC0EF324D96E1B
:10522A00000EF420DA6E000EDF6E00016851010DE7
:10523A00DE0EF324D96E000EF420DA6E000EDF6E55
:10524A000001682BC8D7080E0001D86F040E0001B0
:10525A00D96F160E706E040E0401036F200E026FD2
:10526A00080E0401016F040E0401006F0401008F8F
:10527A00000E556E000E0001E56F12000401205168
:10528A001F0BE806D8A4AAD001D0A8D00401245143
:10529A00D8A4A4D001D0A2D0060E04012119D8B4F2
:1052AA002CD035D02AD05504D8A431D004012451A9
:1052BA00D8A42DD0DE0E0001F76F7D0E0001F86F25
:1052CA00000E0001FC6F090E15D0C00E0001FA6F26
:1052DA001ED05504D8A41BD004012451D8A417D039
:1052EA00D60E0001F76F7C0E0001F86F000E000168
:1052FA00FC6F400EFB6FE9D70AD004012351210A43
:10530A00D8B4D1D7030AD8B4E4D7010A00D004012B
:10531A002039E832030BE806D8A460D04AD05ED020
:10532A0048D05CD07CEC12F059D004012451010D14
:10533A00590EF3240001F76F000EF4200001F86FF4
:10534A00000E0001FC6F010EFB6FC10E20D0800E13
:10535A000001FA6F04012451010D590EF324D96E8C
:10536A00000EF420DA6E23C4DFFF38D00401245182
:10537A00010D580EF3240001F76F000EF42000010E
:10538A00F86F000E0001FC6F010EFB6F810E000129
:10539A00FA6F24D0800E0001FA6F04012451010D26
:1053AA00580EF324D96E000EF420DA6E22C4DFFF01
:1053BA0015D004012151010AD8B410D0030AD8B477
:1053CA00B4D7010AD8B4D2D70A0AD8B4ABD7030AD9
:1053DA00D8B4BDD7010AD8B4DDD700D01200B4D0F2
:1053EA00A5C083F0A6C084F0A7C085F0A8C086F047
:1053FA00A9C087F0AAC088F0F00E0001896F7A0E62
:10540A0000018A6F440E00018B6F7B0E00018C6FC6
:10541A00980E00018D6F7B0E00018E6F2BEC37F01A
:10542A00A5D0A5C083F0A6C084F0A7C085F0A8C007
:10543A0086F0A9C087F0AAC088F04C0E0001896FD7
:10544A00790E00018A6FA00E00018B6F790E0001A0
:10545A008C6FF40E00018D6F790E00018E6F2BECAC
:10546A0037F084D0A5C083F0A6C084F0A7C085F029
:10547A00A8C086F0A9C087F0AAC088F0A40E0001CF
:10548A00896F780E00018A6FF80E00018B6F780E13
:10549A0000018C6FF80E00018D6F780E00018E6F7F
:1054AA002BEC37F063D0A5C083F0A6C084F0A7C068
:1054BA0085F0A8C086F0A9C087F0AAC088F0480E77
:1054CA000001896F7A0E00018A6F9C0E00018B6FB2
:1054DA007A0E00018C6F9C0E00018D6F7A0E00010E
:1054EA008E6F2BEC37F042D0A5C083F0A6C084F0B3
:1054FA00A7C085F0A8C086F0A9C087F0AAC088F026
:10550A00EC0E0001896F7B0E00018A6F400E0001CC
:10551A008B6F7C0E00018C6F400E00018D6F7C0E2C
:10552A0000018E6F2BEC37F021D0A5C07AF0A6C00F
:10553A007BF0A7C07CF0A8C07DF0A9C07EF0AAC00D
:10554A007FF055EC24F012D00001ED51010AD8B4D5
:10555A0068D7030AD8B486D7010AD8B441D7070A4C
:10556A00D8B4A1D7010AD8B4BFD7DFD71200000E2A
:10557A000101976F000E0101986F000E0501086F77
:10558A001E0E096E010E62EC14F0000E016E080E7A
:10559A00026E050E036E010E046E010ED8EC1BF0AE
:1055AA0001C099F102C09AF1FE0EF66E170EF76E5F
:1055BA000900030EF5180900F510D8A43BD0960E81
:1055CA0001013A6F0F0E01013B6F000E0D6E070EBF
:1055DA000D6401D014D00D50010D7C0EF324D96E48
:1055EA00010EF420DA6E0D50010D740EF324E16EF3
:1055FA00010EF420E26EDFCFE7FF0D2AE8D7000E96
:10560A000E6E0B0E0E6401D015D00E50010D5C0EFD
:10561A00F324D96E010EF420DA6E0E50010D500EED
:10562A00F324E16E010EF420E26EDFCFE7FF0E2ACB
:10563A00E8D700D0FE0EF66E170EF76E0900040EBC
:10564A00F55E0900000EF55AD8A06FD0000E0F6E55
:10565A00070E0F6401D028D00F50020D400EF3241C
:10566A00D96E010EF420DA6E0F50020D300EF324BB
:10567A00E16E010EF420E26EDECFE6FFDDCFE5FF3C
:10568A000F50010D840EF324D96E010EF420DA6E48
:10569A000F50010D740EF324E16E010EF420E26E38
:1056AA00DFCFE7FF0F2AD4D7000E106E0B0E10645F
:1056BA0001D028D01050020D180EF324D96E010E15
:1056CA00F420DA6E1050020D000EF324E16E010E82
:1056DA00F420E26EDECFE6FFDDCFE5FF1050010DCC
:1056EA00680EF324D96E010EF420DA6E1050010D03
:1056FA00500EF324E16E010EF420E26EDFCFE7FFD5
:10570A00102AD4D7FE0EF66E170EF76E0900050E94
:10571A00F55E0900000EF55AD8A007D0010E010166
:10572A005A6F020E01015B6F00D0170EC1EC11F027
:10573A0090EC11F001C09DF102C09EF1120004012B
:10574A002205D8A413D0040120511F0B0009D8A4A4
:10575A000DD00001FA8F030E04012119D8A402D03A
:10576A00010E01D0000E0001E36F00D004012251A6
:10577A00D8A431D1040120511F0B020AD8A42BD17D
:10578A00040124510F0B0009D8B425D10401245176
:10579A000F0B196E020E19601ED1200E0001E519B9
:1057AA00D8A419D10001FA8F040124BF1BD0040127
:1057BA0024510F0B196E1950020D370EF324D96EAE
:1057CA00000EF420DA6EDECF1DF0DDCF1EF00401EC
:1057DA0024510F0B196E1950010DDE0EF324D96EE8
:1057EA00000E1AD0040124510F0B196E1950020D24
:1057FA00D80EF324D96E000EF420DA6EDECF1DF037
:10580A00DDCF1EF0040124510F0B196E1950010D42
:10581A00DC0EF324D96E000EF420DA6EDF501C6E13
:10582A0000D01CB002D01D9402D01D8400D0040107
:10583A0024BF0BD0040124510F0B196E1950020D0D
:10584A00370EF324D96E000E0AD0040124510F0B2F
:10585A00196E1950020DD80EF324D96E000EF420D9
:10586A00DA6E1DC0DEFF1EC0DDFF00D0030E04018C
:10587A002119D8A430D01DC0D9FF1EC0DAFFDFAE6F
:10588A001DD0040124BF0BD0040124510F0B196E43
:10589A001950010DDE0EF324D96E000E0AD0040150
:1058AA0024510F0B196E1950010DDC0EF324D96E19
:1058BA00000EF420DA6E0001DF8200D01DC0D9FF8D
:1058CA001EC0DAFF000EDB841DC0D9FF1EC0DAFF3E
:1058DA00000EDB8E80D0040E1D1A1DC0D9FF1EC01B
:1058EA00DAFFDFAE1BD01DC0D9FF1EC0DAFF7F0E64
:1058FA00DF161DC0D9FF1EC0DAFF000EDB8C000EBA
:10590A00126E050E116E1DC013F01EC014F0000EAB
:10591A00166E020E156EBFEC17F007D01DC0D9FF28
:10592A001EC0DAFF000EDB8C00D0040E1D1A1CB25A
:10593A0006D01DC0D9FF1EC0DAFFDFAE32D0040187
:10594A0024BF0BD0040124510F0B196E1950010DFD
:10595A00DE0EF324D96E000E0AD0040124510F0B77
:10596A00196E1950010DDC0EF324D96E000EF420C5
:10597A00DA6E0001DF9200D01DC0D9FF1EC0DAFF27
:10598A003B0EDF16000E126E050E116E1DC013F0CF
:10599A001EC014F0000E166E020E156EBFEC17F044
:1059AA0007D01DC0D9FF1EC0DAFF3B0EDF1600D09C
:1059BA00040124510F0B196E1950010D700EF324B6
:1059CA001A6E0F0EF4201B6E1AC0D9FF1BC0DAFF25
:1059DA00FE0EDF1600D012000001816FA10E000139
:1059EA00816193D081C060F00001616B000E0001FB
:1059FA00636F070E626FC9EC1DF0D8900001603723
:105A0A00000161374A0E0001602500017F6F7D0E9B
:105A1A00000161210001806F000E0001826F22D017
:105A2A0000018251010D7FC07AF080C07BF0F350F3
:105A3A0000017A27F45000017B237AC0F6FF7BC06D
:105A4A00F7FF00018251010DF35000017825D96E4C
:105A5A00F45000017921DA6E0800F5CFDFFF00016A
:105A6A00822B00D0020E0001826118D000018251FF
:105A7A00010D7FC07AF080C07BF0F35000017A27D5
:105A8A00F45000017B237AC0F6FF7BC0F7FF0800C1
:105A9A00F5500009D8B402D0C3D700D081C060F055
:105AAA000001616B000E0001636F070E626FC2ECAA
:105ABA001AF06D0E00016025F66E770E0001612165
:105ACA00F76E00018251010DF35000017825D96E5D
:105ADA00F45000017921DA6E0800F5CFDFFF0DD00E
:105AEA0000018251010DF35000017825D96EF4505E
:105AFA0000017921DA6E000EDF6E0001822B00D0E0
:105B0A00020E00018265ECD713D1A00E0001816557
:105B1A002AD0B70E0001816126D078C06EF079C014
:105B2A006FF05F0E000181250001686F0001696B4B
:105B3A00FF0E6923000E00016B6F030E6A6F0CECF7
:105B4A0014F0940E000168250001706F7C0E0001AC
:105B5A0069210001716F000E0001736F030E726FED
:105B6A00EEEC16F0E5D0C70E000181653AD0E20EE0
:105B7A000001816136D078C06EF079C06FF0700E86
:105B8A0000017A6FFE0E00017B6F00018151000156
:105B9A007C6F7D6BD89000017C377D3700017A518C
:105BAA0000017C2700017B5100017D23160E0001B4
:105BBA007C250001706F7D0E00017D210001716F4F
:105BCA00000E0001736F020E726FEEEC16F0000108
:105BDA0020EE02F07851D9267951DA22000EDF6ED2
:105BEA00A7D0E50E0001816593D0F20E0001816114
:105BFA008FD0000181511A0F0001826F28D0000155
:105C0A008251030D8A0EF32400017F6F7E0E1BD092
:105C1A0000018251030D420EF32400017F6F7E0EB4
:105C2A0012D000018251030D660EF32400017F6F2A
:105C3A007E0E09D000D000018251030DF60EF32426
:105C4A0000017F6F7E0EF4200001806F0FD00001EB
:105C5A00E951000AD8B4EFD7010AD8B4E2D7030A47
:105C6A00D8B4CDD7010AD8B4D3D7E5D7000E0001EE
:105C7A00826F020E0001826501D05AD00001825162
:105C8A00010D7FC07AF080C07BF0F35000017A27C3
:105C9A00F45000017B237AC0F6FF7BC0F7FF0800AF
:105CAA00F5CF7EF090EC12F00009D8A40ED01FD0E8
:105CBA000CD0300E07D0320E05D02E0E03D0250E92
:105CCA0001D0260E00017E6F12D000017E51260AF5
:105CDA00D8B4F5D7010AD8B4F4D7080AD8B4E9D7A2
:105CEA001F0AD8B4E8D7050AD8B4E7D700D000010C
:105CFA008251010DF35000017825D96EF45000014C
:105D0A007921DA6E7EC0DFFF0001822BB2D710D074
:105D1A0078C060F079C061F0000E0001636F000E78
:105D2A00626F000E0001656F030E646FD6EC13F00C
:105D3A001200ABC060F0ACC061F0ADC062F0AEC0A2
:105D4A0063F0000E0001656F080E646FB4EC18F082
:105D5A000001605100016111D8A402D0000EAFD138
:105D6A00AFC060F0B0C061F0000E0001636F000EBA
:105D7A00626F000E0001656F080E646FD6EC13F0B7
:105D8A00000120EE01F0AB51D926AC51DA22000114
:105D9A00DFA04BD1ABC0D9FFACC0DAFFDF500001A6
:105DAA00B56F020E0001B76F010E0001BB6F020E44
:105DBA000001B86F26D10001B8510001686F696B04
:105DCA0068BF6907000E00016B6F010E6A6F0CEC69
:105DDA0014F0000168510001AB25D96E0001695128
:105DEA000001AC21DA6EDF500001B66F0001B65136
:105DFA00D1EC20F06EC0B3F06FC0B4F0000E000119
:105E0A00B96FF1D00001B9510001686F696B68BFC1
:105E1A006907000E00016B6F010E6A6F0CEC14F03B
:105E2A00B3C0B1F0B4C0B2F0000168510001B127AB
:105E3A00000169510001B223B1C0F6FFB2C0F7FFF9
:105E4A000800F5CFBAF0020E0001AD250001606F1F
:105E5A00000E0001AE210001616FB6C062F00001C0
:105E6A00636B000E0001656F060E646F89EC17F014
:105E7A000001605100016111D8A402D0010E01D0C5
:105E8A00000E0001BC6F7FD0ABD00001BC510001F5
:105E9A00D8B4A6D0E5EC24F047D0A2D00001BC517A
:105EAA000001D8B49DD074EC13F03ED099D0000113
:105EBA00BC510001D8B494D0E4EC12F035D090D0A3
:105ECA000001BC510001D8B48BD02CEC13F02CD0BB
:105EDA0087D00001BC510001D8B482D0FCEC12F08A
:105EEA0023D07ED00001BC510001D8B479D05CEC3B
:105EFA0013F01AD075D00001BC510001D8B470D08B
:105F0A0014EC13F011D06CD00001BC510001D8B4CC
:105F1A0067D044EC13F008D063D00001BC510001F3
:105F2A00D8B45ED08CEC13F0040E0001BB6F58D0CD
:105F3A000001B58155D00001B58952D00001B58361
:105F4A004FD00001B58B4CD0ABC0D9FFACC0DAFF43
:105F5A00DF500001686FBCC069F00001BA5131EC32
:105F6A0018F00001BA6F0001B751010DF35000019A
:105F7A00AF25D96EF4500001B021DA6EBAC0DFFF46
:105F8A000001B72B2DD00001BA51000AD8B428D08D
:105F9A003A0AD8B47AD7010AD8B480D7070AD8B44B
:105FAA0086D7010AD8B48CD7030AD8B492D7010A83
:105FBA00D8B498D77F0AD8B49ED7010AD8B4A4D740
:105FCA00030AD8B4AAD7A20AD8B4B2D7010AD8B455
:105FDA00B5D7050AD8B4AFD7010AD8B4B2D7B4D75F
:105FEA000001B92B00D00001B951800A7D0FD8B049
:105FFA0005D0070E0001B76505D700D00001B82B00
:10600A0000D00001B851800A780FD8B007D0040E2A
:10601A000001BB19D8B402D0CED600D0AFC0D9FF88
:10602A00B0C0DAFFB5C0DFFF29D0ABC060F0ACC0AA
:10603A0061F0F7EC17F00009D8B40FD0ABC0A5F0A7
:10604A00ACC0A6F0ADC0A7F0AEC0A8F0AFC0A9F032
:10605A00B0C0AAF0F4EC29F00ED0ABC07AF0ACC014
:10606A007BF0ADC07CF0AEC07DF0AFC07EF0B0C0BA
:10607A007FF055EC24F00001BB6F00D00001BB0596
:10608A00D8B40AD0030E0001BB19D8B405D0040E47
:10609A000001BB19D8A410D0ADC06EF0AEC06FF02D
:1060AA00ABC070F0ACC071F0000E0001736F080E47
:1060BA00726FC0EC21F000D00001BB5100D0120079
:1060CA00000E0001C16F78EC1FF00009D8B410D09F
:1060DA007BD10ED00001E651010DCF0EF324D96E0B
:1060EA00010EF420DA6E0E0EDF6E0001E62B00D0F0
:1060FA000001E651800A780FD8A0ECD70001E851D8
:10610A00060D9F0EF32400016E6F010EF4200001AC
:10611A006F6FD10E0001706F010E0001716F000EDA
:10612A000001736F060E726FC0EC21F0EEC0CFF162
:10613A000001EBA503D00101D08100D00001F55187
:10614A00D8B423D0CF0E0001606F010E0001616F39
:10615A00F7EC17F00009D8B418D00001F451010186
:10616A00CF130001EFB307D00001EEA304D0020E53
:10617A000001F41B00D00001EFBB07D00001EEAB19
:10618A0004D0200E0001F41B00D0EEC0EFF0000195
:10619A00E75100080001E825060F0001C36F00015E
:1061AA00C351800A7A0FD8A003D0FA0E0001C32780
:1061BA000001C351050F0001C56F0001C551800AD6
:1061CA007A0FD8A004D0FA0E0001C52700D0020E1B
:1061DA000001E66F000E0001C46F0001C451800A7D
:1061EA007A0FD8B05BD001D059D00001C351060D47
:1061FA009F0E0001BF6F010E0001C06FF350000136
:10620A00BF27F4500001C0230001C451010DF3500F
:10621A000001BF25D96EF4500001C021DA6EDF50AB
:10622A000001C26F0001C551060D9F0EF324000143
:10623A00606F010EF4200001616FC2C062F00001BC
:10624A00636B000E0001656F060E646F89EC17F030
:10625A000001605100016111D8B40ED00001E6516D
:10626A00010DCF0EF324D96E010EF420DA6EC2C0EE
:10627A00DFFF0001E62B00D00001C42BAED70ED001
:10628A000001E651010DCF0EF324D96E010EF42060
:10629A00DA6E0E0EDF6E0001E62B00D00001E65129
:1062AA00800A780FD8A0ECD7CF0E0001606F010EDC
:1062BA000001616FD70E0001626F010E0001636F6A
:1062CA00000E0001656F080E646FB4EC18F000014F
:1062DA00605100016111D8B470D0D10E0001606F15
:1062EA00010E0001616FD90E0001626F010E0001FB
:1062FA00636F000E0001656F060E646FB4EC18F050
:10630A000001605100016111D8A410D00E0E0101E4
:10631A00D119D8B40BD00101D051D8A407D0CFC11C
:10632A00BFF0220E0001BF17D8B41CD00E0E010117
:10633A00D119D8B404D0000E0001F46F00D0CF0EEA
:10634A000001AB6F010E0001AC6FD70E0001AD6FFB
:10635A00010E0001AE6FBDC0AFF0BEC0B0F09EEC42
:10636A002EF028D00101D851D8B404D00101D0515F
:10637A00D8B423D00101D7A303D00101CFA31DD0E4
:10638A000101D7AB05D00101CFAB17D001D015D091
:10639A00CF0E0001AB6F010E0001AC6FD70E0001EA
:1063AA00AD6F010E0001AE6FBDC0AFF0BEC0B0F060
:1063BA009EEC2EF00001C16F00D0BDC07AF0BEC0C5
:1063CA007BF0FFEC33F02DD00001E851050F0001FE
:1063DA00C56F0001C551800A7A0FD8A004D0FA0E01
:1063EA000001C52700D00001E851060D9F0EF324D5
:1063FA0000016E6F010EF42000016F6F0001C5519C
:10640A00060D9F0EF3240001706F010EF4200001A7
:10641A00716F000E0001736F060E726FC0EC21F0EF
:10642A0000D00001E82B0001E851800A7A0FD8A0B9
:10643A0003D0000E0001E86F020E0001E66F000EA5
:10644A000001EE6F000E0101D06F0001C15100D0B2
:10645A001200020E0001FD19D8B43BD0030E000150
:10646A00FD19D8A402D035D000D09DC1C6F09EC176
:10647A00C7F00001C61FC71FC64BC72B99EC11F006
:10648A000001C651000160270001C75100016123C4
:10649A00000161BFEAD70001615107E18D0E0001D9
:1064AA00605DD8B002D0E1D700D099EC11F060C09D
:1064BA009DF161C09EF10001E02BE0C0C6F0000131
:1064CA00C76BC6BFC7070001C6B193D102D091D12D
:1064DA0000D00101975101019811D8B413D097C186
:1064EA00D9FF98C1DAFF0101DFAE04D00001C66B03
:1064FA00C62B02D00001C66B0001C6510001C96F4C
:10650A00CA6B06D0000E0001CA6F000EC96F00D018
:10651A000001C9510001CA11D8A432D1030E0001E9
:10652A00FD19D8A41AD005010251D8B40AD0A4EC96
:10653A0012F005010219D8A404D0000E0501026F59
:10654A0006D12BEC15F00501026F05010251D8A402
:10655A00FED0000E0001FD6FFAD0070E0001CF6FCA
:10656A0079D00001CF51010D740EF324D96E010EBA
:10657A00F420DA6EDF50FF0A0001C66F0001CF5126
:10658A00020D300EF324D96E010EF420DA6EDECF3E
:10659A00C7F0DDCFC8F0C7C0D9FFC8C0DAFF000115
:1065AA00C651DF16000E0001CE6F0B0E0001CE653C
:1065BA0001D02DD00001CE51010D500EF324D96E19
:1065CA00010EF420DA6EDF500001C66F0001CE51D1
:1065DA00020D000EF324D96E010EF420DA6EDECF1E
:1065EA00C7F0DDCFC8F0C7C0D9FFC8C0DAFFDF5097
:1065FA000001C6150009D8A407D0CEC07AF0000160
:10660A00CF51C9EC23F000D00001CE2BCED7000128
:10661A00CF51010D740EF324D96E010EF420DA6EF7
:10662A00DF500001C66F0001CF51020D300EF32476
:10663A00D96E010EF420DA6EDECFC7F0DDCFC8F0D6
:10664A00C7C0D9FFC8C0DAFF0001C651DF12000176
:10665A00CF0700D00001CFAF84D7000E0001BD6F75
:10666A00050E0001BE6F65EC30F00001FD6F60D0D1
:10667A00100E0001606F050E0001616F000E00012F
:10668A00636F000E626F000E0001656F060E646F85
:10669A00D6EC13F05CD0000E0001CD6F050E0001A0
:1066AA00CD6501D00FD00001CD51010D020EF324AA
:1066BA00D96E050EF420DA6EDF5050EC15F00001A9
:1066CA00CD2BECD7060EB6EC11F00501026F030EC6
:1066DA000001606F050E0001616F000E0001636F1B
:1066EA00000E626F000E0001656F050E646FD6EC36
:1066FA0013F02DD0030E0001FD6F000E0501006F8F
:10670A00800EB6EC11F00501026F030E0001606FF6
:10671A00050E0001616F000E0001636F000E626FCB
:10672A00000E0001656F050E646FD6EC13F00FD0F2
:10673A000001FD51010AD8B40AD0030AD8B498D787
:10674A00010AD8B4A8D7070AD8B4D4D700D0000110
:10675A00FD510001D8B414D0010E0001606F000E83
:10676A000001616F050E0001626F080E0001636F80
:10677A00010E09EC1FF060C097F161C098F100D0DA
:10678A000101995101019A11D8B413D099C1D9FFC5
:10679A009AC1DAFF0101DFAE04D00001C66BC62B35
:1067AA0002D00001C66B0001C6510001CB6FCC6B51
:1067BA0006D0000E0001CC6F000ECB6F00D0000196
:1067CA00CB510001CC11D8A414D0000E0001606F87
:1067DA00080E0001616F050E0001626F010E0001D3
:1067EA00636F010E09EC1FF060C099F161C09AF164
:1067FA0000D01200020E0001806F00018051800A51
:10680A00780FD8B022D303D320D301D346D00001C6
:10681A0080510001686F696B68BF6907000E00014B
:10682A006B6F010E6A6F0CEC14F0000168510001E5
:10683A007A25D96E0001695100017B21DA6E680E52
:10684A002AD0000180510001686F696B68BF69072F
:10685A00000E00016B6F010E6A6F0CEC14F0000160
:10686A00685100017A25D96E0001695100017B2126
:10687A00DA6E690E10D000D0000180510001686FF5
:10688A00696B68BF6907000E00016B6F010E6A6FC2
:10689A000CEC14F073D1DF6ED5D2000180510001E7
:1068AA00686F696B68BF6907000E00016B6F010EA4
:1068BA006A6F0CEC14F00001685100017A25D96E58
:1068CA000001695100017B21DA6EDF508A0AD8B4CF
:1068DA00D3D7010AD8B4D0D71B0AD8B498D7010A9B
:1068EA00D8B4AFD7AFD281D000D000018051000117
:1068FA00686F696B68BF6907000E00016B6F010E54
:10690A006A6F0CEC14F03AD1020E0001EC19D8B4FB
:10691A0005D0050E0001EC19D8A494D27AC0D9FF8B
:10692A007BC0DAFF000EDB84000180510001686F32
:10693A00696B68BF6907000E00016B6F010E6A6F11
:10694A000CEC14F00001685100017A2500016E6F09
:10695A000001695100017B2100016F6F0001805124
:10696A000001686F696B68BF6907000E00016B6FF1
:10697A00010E6A6F0CEC14F07AC07CF07BC07DF0DB
:10698A000001685100017C270001695100017D2343
:10699A00010E00017C250001706F000E00017D21AF
:1069AA000001716F80C07EF000017F6B7EBF7F07A0
:1069BA0000017E1F7F1F7E4B7F2B070E00017E2565
:1069CA000001726F000E00017F210001736FC0EC9D
:1069DA0021F0000120EE07F07A51D9267B51DA2204
:1069EA00000EDF6E000180072DD2000180510001E8
:1069FA00686F696B68BF6907000E00016B6F010E53
:106A0A006A6F0CEC14F00001685100017A25D96E06
:106A1A000001695100017B21DA6EDF50650AD8B4A2
:106A2A0073D7EF0AD8B461D7010AD8B45ED70AD2AD
:106A3A004DD0000180510001686F696B68BF69071A
:106A4A00000E00016B6F010E6A6F0CEC14F000016E
:106A5A00685100017A25D96E0001695100017B2134
:106A6A00DA6E2C0EF3D07AC0D9FF7BC0DAFF030EA0
:106A7A00DF12E8D1000180510001686F696B68BFBD
:106A8A006907000E00016B6F010E6A6F0CEC14F0BF
:106A9A000001685100017A25D96E0001695100018F
:106AAA007B21DA6E2A0ED2D0DED700D000018051C7
:106ABA000001686F696B68BF6907000E00016B6FA0
:106ACA00010E6A6F0CEC14F059D0BCD10001805150
:106ADA000001686F696B68BF6907000E00016B6F80
:106AEA00010E6A6F0CEC14F00001685100017A255E
:106AFA00D96E0001695100017B21DA6EDF508A0AE2
:106B0A00D8B4D4D7010AD8B4D1D71B0AD8B491D7EC
:106B1A00010AD8B4AFD796D13ED000D00001805137
:106B2A000001686F696B68BF6907000E00016B6F2F
:106B3A00010E6A6F0CEC14F00001685100017A250D
:106B4A00D96E0001695100017B21DA6E350EF9D048
:106B5A007AC0D9FF7BC0DAFF000EDB8473D100D084
:106B6A00000180510001686F696B68BF6907000EF8
:106B7A0000016B6F010E6A6F0CEC14F00001685192
:106B8A0000017A25D96E0001695100017B21DA6E74
:106B9A002C0E81D657D1000180510001686F696BB4
:106BAA0068BF6907000E00016B6F010E6A6F0CEC7B
:106BBA0014F00001685100017A25D96E000169516B
:106BCA0000017B21DA6EDF508A0AD8B4C9D7010ADC
:106BDA00D8B4C6D71B0AD8B4A1D7010AD8B49ED74D
:106BEA0031D137D0000180510001686F696B68BFED
:106BFA006907000E00016B6F010E6A6F0CEC14F04E
:106C0A000001685100017A25D96E0001695100011D
:106C1A007B21DA6E8A0E1AD026D700018051000134
:106C2A00686F696B68BF6907000E00016B6F010E20
:106C3A006A6F0CEC14F00001685100017A25D96ED4
:106C4A000001695100017B21DA6E8B0EDF6E0BD7D2
:106C5A00F9D0000180510001686F696B68BF69074C
:106C6A00000E00016B6F010E6A6F0CEC14F000014C
:106C7A00685100017A25D96E0001695100017B2112
:106C8A00DA6EDF50900AD8B4ADD7010AD8B4C5D7A6
:106C9A00D9D01CD000D0000180510001686F696B07
:106CAA0068BF6907000E00016B6F010E6A6F0CEC7A
:106CBA0014F00001685100017A25D96E000169516A
:106CCA0000017B21DA6E350EE6D5BCD00001805179
:106CDA000001686F696B68BF6907000E00016B6F7E
:106CEA00010E6A6F0CEC14F00001685100017A255C
:106CFA00D96E0001695100017B21DA6EDF50900ADA
:106D0A00D8B4C9D7010AD8B4C6D79CD01DD000D0F0
:106D1A00000180510001686F696B68BF6907000E46
:106D2A0000016B6F010E6A6F0CEC14F000016851E0
:106D3A0000017A25D96E0001695100017B21DA6EC2
:106D4A002C0EDF6E05D77ED0000180510001686FDE
:106D5A00696B68BF6907000E00016B6F010E6A6FED
:106D6A000CEC14F00001685100017A25D96E00017B
:106D7A00695100017B21DA6EDF50900AD8B4C8D776
:106D8A00010AD8B4C5D75ED022D000D00001805104
:106D9A000001686F696B68BF6907000E00016B6FBD
:106DAA00010E6A6F0CEC14F00001685100017A259B
:106DBA00D96E0001695100017B21DA6E2C0EDF6E5B
:106DCA007AC0D9FF7BC0DAFF000EDB823BD000011C
:106DDA0080510001686F696B68BF6907000E000186
:106DEA006B6F010E6A6F0CEC14F000016851000120
:106DFA007A25D96E0001695100017B21DA6EDF50D4
:106E0A00900AD8B4C3D7010AD8B4C0D71BD000019E
:106E1A00F251000AD8B441D5010AD8B4E6D5030A1A
:106E2A00D8B454D6010AD8B4B6D6070AD8B411D7FA
:106E3A00010AD8B44BD7030AD8B486D7010AD8B402
:106E4A00C6D700D00001802BD8D4120083C0D9FF46
:106E5A0084C0DAFFDF5000019F6F020E0001A46FA9
:106E6A00010E0001916F83C0D9FF84C0DAFFDF50A1
:106E7A00DD0B0001966F87C0D9FF88C0DAFF96C084
:106E8A00DFFF020E0001956FEED20001955100015D
:106E9A00686F696B68BF6907000E00016B6F010EAE
:106EAA006A6F0CEC14F00001685100018325D96E59
:106EBA000001695100018421DA6EDF500001A16FDF
:106ECA00A1C060F00001616B000E0001636F0C0E3F
:106EDA00626FC9EC1DF0000160510001A06FA1C0F2
:106EEA0060F00001616B000E0001636F0C0E626FAF
:106EFA00C2EC1AF0000160510001976F0001A15124
:106F0A0070EC1AF00001A36F0001A3510001D8B47C
:106F1A002AD00001A451010DF35000018725D96E32
:106F2A00F45000018821DA6EA3C0DFFF0001A42B10
:106F3A00520E0001606F000E0001616F000E000129
:106F4A00636F000E626F000E0001656F030E646FBF
:106F5A00D6EC13F019D183C0D9FF84C0DAFFDF5011
:106F6A000001966F7DD2000E0001926F00019F51C1
:106F7A00220B220AD8A40FD04CA203D000019F935F
:106F8A000AD085C0D9FF86C0DAFF0001DFAA03D084
:106F9A0000019F9B00D0060E0001A06504D0000EE0
:106FAA000001A26F34D000019FA308D00001A051B4
:106FBA000C0D8BC08FF08CC090F012D000019FABEB
:106FCA0008D00001A0510C0D8DC08FF08EC090F03A
:106FDA0007D00001A0510C0D89C08FF08AC090F033
:106FEA00F35000018F27F4500001902300019751BC
:106FFA00010DF35000018F27F450000190238FC038
:10700A00F6FF90C0F7FF0800F5CFA2F000D000010C
:10701A00A2510001D8B445D0D00E0001A26505D016
:10702A00E00E0001A2653DD000D0010E0001926F72
:10703A00020E0001986F00019851800A780FD8B0AB
:10704A0030D001D02ED0000198510001686F696BD1
:10705A0068BF6907000E00016B6F010E6A6F0CECC6
:10706A0014F00001685100018525D96E00016951AB
:10707A0000018621DA6E0001A151DE18D8A40DD0D4
:10708A000E0E0001A16F010E0001A06F020E000199
:10709A00976F000E0001A26F04D00001982BCBD786
:1070AA0000D00001A2510001D8B40BD09C0E0001FF
:1070BA00786F000E0001796F0001A251F1EC2CF0FB
:1070CA0000D00001A2510001D8B405D000019C51A2
:1070DA000001D8A461D00001A15141EC23F00001C4
:1070EA00A36F0001A3510001D8B4BAD183C0D9FF5C
:1070FA0084C0DAFFDF500001686F020E00018525A7
:10710A000001606F000E000186210001616FA3C0BB
:10711A0062F00001636B000E0001656F060E646F7A
:10712A0089EC17F00001605100016111D8A402D066
:10713A00010E01D0000E0001696F0001A35131EC6C
:10714A0018F00001A36F0001A451010DF3500001D2
:10715A008725D96EF45000018821DA6EA3C0DFFFBB
:10716A000001A42B520E0001606F000E0001616F36
:10717A00000E0001636F000E626F000E0001656F62
:10718A00030E646FD6EC13F083C0D9FF84C0DAFF14
:10719A00DF504C6EE0D664D1000192510001D8B4A0
:1071AA0060D0000E0001996F48D0000E00019A6F5E
:1071BA002DD000019A51010D9C0EF324D96E000EB8
:1071CA00F420DA6E00019951010DE70EF324E16E05
:1071DA00010EF420E26EDE50E618D8A414D0E70EB1
:1071EA000001606F010E0001616F000E0001636F04
:1071FA00000E626F000E0001656F030E646FD6EC1D
:10720A0013F0020E79D100019A2B00D000019A5195
:10721A00800A7D0FD8B00ED000019A51010D9C0E44
:10722A00F324D96E000EF420DA6EDF50D8B402D0FF
:10723A00C0D700D00001992B00D000019951800AD3
:10724A007D0FD8B00ED000019951010DE70EF3243D
:10725A00D96E010EF420DA6EDF50D8B402D0A5D769
:10726A0000D0030E0001916F000E00019B6FC7D082
:10727A0000019B51010D9C0EF324D96E000EF420DF
:10728A00DA6EDF500001A36FA8D05250D8B4B4D040
:10729A00F60E0001606F7F0E0001616F52C062F04E
:1072AA000001636B000E0001656F040E646F89ECC8
:1072BA0017F060C093F061C094F00001935100018F
:1072CA009411D8B499D0060E0001A46195D000019A
:1072DA00A451010DF35000018725D96EF450000125
:1072EA008821DA6E2A0EDF6E0001A42BF60E000149
:1072FA008F6F7F0E0001906F00018F1F901F8F4BC1
:10730A00902B0001935100018F2700019451000135
:10731A0090237A0E00018F25F66E770E9021F76E74
:10732A000001A451010DF35000018725D96EF450D4
:10733A0000018821DA6E0800F5CFDFFF33D00001A3
:10734A00A451010DF35000018725D96EF4500001B4
:10735A008821DA6E53C0DFFF28D04ED00B0E5218A8
:10736A00D8A44AD0060E0001A46146D00001A45157
:10737A00010DF35000018725D96EF45000018821D0
:10738A00DA6E2A0EDF6E0001A42B0001A451010D52
:10739A00F35000018725D96EF45000018821DA6E76
:1073AA00130EDF6E0001A42BCAD70001A42B24D030
:1073BA000001968321D00001968B1ED00001A451B2
:1073CA00010DF35000018725D96EF4500001882180
:1073DA00DA6EA3C0DFFFE9D70FD00001A351E10A9B
:1073EA00D8B4E6D7040AD8B4E6D7160AD8B44DD723
:1073FA00070AD8B4B3D7E2D700019B2B00D000010B
:10740A009B51800A7D0FD8B011D000019B51010D0C
:10741A009C0EF324D96E000EF420DA6EDF50D8B435
:10742A0005D0070E0001A46523D700D0520E000133
:10743A006E6F000E00016F6F9C0E0001706F000EE0
:10744A000001716F000E0001736F030E726FEEEC94
:10745A0016F083C0D9FF84C0DAFFDF504C6E00D02B
:10746A000001952B00D000019551800A780FD8B001
:10747A0005D0070E0001A46508D500D0020E000150
:10748A00A4651AD0E70E00016E6F010E00016F6F3E
:10749A00520E0001706F000E0001716F000E0001A4
:1074AA00736F030E726FEEEC16F087C0D9FF88C0B7
:1074BA00DAFF96C0DFFF1DD0E70E0001606F010EF4
:1074CA000001616F000E0001636F000E626F000E13
:1074DA000001656F030E646FD6EC13F083C0D9FF09
:1074EA0084C0DAFF87C0E1FF88C0E2FFDFCFE7FF91
:1074FA0000D00001915100D01200000D01020304D6
:10750A0005060708090A1624000E0E0E0E0E0E0EA8
:10751A000E0B2F54180E0E0E41420E0E0E235F55FF
:10752A000C0E0E0E4D4E0E0E0E175E561925262700
:10753A00282B2C2D2E225D573031323334373839EF
:10754A003A3B5C583C3D3E3F4043444546475B59C5
:10755A0048494A4B4C4F505152535A2F3B3C3D3E9F
:10756A003F40414243442E353A00000000000000EB
:10757A00004531301E0000000000000000272D2ABF
:10758A001F20212200002324252634141A09130A55
:10759A0000000D0F181C33041516170729650B1167
:1075AA00080C121D1B0619052B280E10363738E059
:1075BA00E3F0E12CE2E62CE5F0E7E42F3B3C3D3E2C
:1075CA003F404142434431353A0000000000000088
:1075DA0000452E301E000000000000000027383948
:1075EA001F2021220000232425262D343637131C80
:1075FA000000090A06150F041208180C2965070B62
:10760A0017111633140D0E1B2B2805101A191DE01D
:10761A00E3F0E12AE2E62CE5F0E7E4303B3C3D3ECC
:10762A003F40414243442E893A00000000000000D6
:10763A0000452F321E0000000000000000272D39EF
:10764A001F20212200002324252634141A08151786
:10765A0000001C180C1213041607090A29650B0DE1
:10766A000E0F331D1B0619052B281110363738E06B
:10767A00E3F0E12AE2E62CE5F0E7E4303B3C3D3E6C
:10768A003F40414243442D893A0000000000000077
:10769A0000452F321E000000000000000027342E93
:1076AA001F2021220000232425262A141A08151730
:1076BA0000001C180C1213041607090A29650B0D81
:1076CA000E0F331D1B0619052B281110363738E00B
:1076DA00E3F0E158E2E62CE5F0E7E42F3B3C3D3EDF
:1076EA003F40414243442E353A000000000000006A
:1076FA00004531301E0000000000000000272D392F
:10770A001F20212200002324252634141A081517C5
:10771A0000001C180C1213041607090A29650B0D20
:10772A000E0F331D1B0619052B281110363738E0AA
:10773A00E3F0E12AE2E62CE5F0E7E40000000000CD
:10774A0000000000000000005500FB006754000024
:10775A005F606156005C5D5E5700595A5B280062A3
:10776A0000630000040C1808121CFA7F367FA27D01
:10777A000A1D070540383028CC7D4900003B00002F
:10778A003C00003D00003E00003F00004000004178
:10779A0000004200007F0000810000480000E04C29
:1077AA00003A000000000000000000000000000095
:1077BA0000000000000000000000000080000047F8
:1077CA000000E0E11DE01E000000000000000000D3
:1077DA00000000000000000000000000000000009F
:1077EA00E027004600004C0000E01F00E02000E017
:1077FA002100E02200000000000000E02300E0E198
:10780A0050E15200E0E14F530000E01400E01A009A
:10781A004B0000E01500E01700000000000000E047
:10782A004A00E05000520000E04F00E04D00E00442
:10783A0000E016004E0000E00900E00A00290000FE
:10784A003900004A00005000005100004F00004D6E
:10785A000000E01D00E01B00E00600E019009100B6
:10786A00002B0000280000900000E15000E15100C8
:10787A00E14F00E14D0000000000000000000000A0
:10788A000000E02A00000000000000E02C000000D8
:10789A0000000000000000000000000000000000DE
:1078AA0000000000000000000000000000000000CE
:1078BA0000000000000000000000000000000000BE
:1078CA0000000000000000000000B69AB5B4B30042
:1078DA00002A31383F4604030201050000070E154D
:1078EA001C23AE6993A4B200004D545BCD62000024
:1078FA00000000000000000000000000000000007E
:10790A00000000000000000000000000000000006D
:10791A000000000000000000000000000000ACA908
:10792A00A6A2B00000307A3EC84CABA8A5A1AF0011
:10793A00000D141B2229ADAAA7A3B10000535A6156
:10794A00CE68E600000000000000000000CA000047
:10795A0000000000000000000000E7000000000036
:10796A000000000000CD0000000000000000000040
:10797A000000CE08160C0F000039170A18CD0310A4
:10798A00190B120000241A0902C8CE251126270055
:10799A00002E132028ECE600000000000000000082
:1079AA0000CA000000000000000000000000E7CC50
:1079BA00000000000000000000CD00EDF1E6E70045
:1079CA0000EAEB0000006A043A7F3C0000475D5081
:1079DA005E4844011D812F000063604F4BC86CC98B
:1079EA003D326B000049594A67ECE800000000008C
:1079FA000000000000CB00000000000000000000B2
:107A0A000000E9CC000000000000000000CD00EDFD
:107A1A00F1E6E70000EAEB000000CE4E5C525500AA
:107A2A0000361E3B2B6D96565F515800002C0521DF
:107A3A00837ACE6457656600001F342D406ED300EA
:107A4A00000000000000000000000000000000002C
:107A5A00000000000000D4D7000000000000000071
:107A6A0000DE0000000000000000000000DD000051
:107A7A00000000000000000000D10000000000002B
:107A8A000000000000000000DB0000000000000011
:107A9A0000E0D30000000000000000000000000029
:107AAA0000000000000000000000D40000000000F8
:107ABA000000000000DE00000000000000000000DE
:107ACA0000DF000000B300000000000000D2000048
:107ADA0046D6D5000000D9D8DC000000000000001E
:107AEA000000DA000000E6000000000000000000CC
:107AFA000000000000000000000000000000E70095
:107B0A00000000000000000000000000000000006B
:107B1A00000000000000393B0C2483000009210A00
:107B2A00013C161A08192F000044020310C82B3A08
:107B3A001E0F1D00001118CDCE7AE60000000000CD
:107B4A00000000000000EE0000000000000000003D
:107B5A000000E70000000000000000000000000034
:107B6A00000000000000000000002513EC7F280040
:107B7A00004F5150CC8E1F208136260000CA5D96D8
:107B8A0056906D6E1234270000575EEFF086E800BB
:107B9A0000000000000000000000000000000000DB
:107BAA00000000000000E9000000000000000000E2
:107BBA0000000000000000000000000000006459FE
:107BCA005263670000040B2E2D3D5C604E5F65001A
:107BDA00000517C92C3271745855660000406B6A4B
:107BEA00CB6CE6000000000000000000000000006E
:107BFA0000000000000000000000E7000000000094
:107C0A000000000000170000000000000000000053
:107C1A00001D130B121983000018C821443A2408C6
:107C2A00101A1600000A0302CA09110C1E0F0100DD
:107C3A00007A3BCDCE3CE8000000000000000000C6
:107C4A000000000000000000000000000000E90041
:107C5A00000000000000000000E600000000000034
:107C6A000000000000E76ACB28262E000025042C1D
:107C7A00321F6B2739813600002B052F40346C6D7B
:107C8A006E207F00002D3DECC9CC041111040E18A2
:107C9A00041718040C000C11110C0E180C171818E4
:107CAA001111180E18181718081111080E0C0817B8
:107CBA0018080C00121111120E18121718121800B7
:107CCA000600000900000D00001400000501090665
:107CDA00A101050719E029E7150025017501950895
:107CEA008102950175088103950575010508190139
:107CFA0029059102950175039103950675081500EA
:107D0A0026FF000507190029FF8100C011112D0067
:107D1A00F300F400E13836003700E136E1372F008E
:107D2A003000E130E13234002E002D001E00380010
:107D3A003200E1278700E136E137E1388900E11EA8
:107D4A0000000E001600170011000B0010001C00A6
:107D5A0015001A0013000A001D00070005001B0089
:107D6A001B0E1B171B1C1B1A1A1C19000F00E0E123
:107D7A00E3E2E6E5E4E0E1E29190E5E4E0E1E391C3
:107D8A0090E5E4E1E0E3E2E6E4E5E1E0E29190E4B3
:107D9A00E5E1E0E39190E4E52A034500730072000F
:107DAA0069006C006C00650020004E0065007700D9
:107DBA0020004B006500790062006F0061007200CC
:107DCA00640009022900010100A03209040000022E
:107DDA000301010009211101000122400007058168
:107DEA000308000107050103080001130628000023
:107DFA0010040628001E272104281E272105281EF4
:107E0A00272604281E27260528042D161328162D92
:107E1A001613280612131C150C0A0B172C1F271EE3
:107E2A00202D1F271E222C0816150C0F0F082C0CAC
:107E3A0011063728091F2C002F0000300000E12FFF
:107E4A0000E13000E2E126E2E127380000380000D4
:107E5A00383838360000370000E135002F0000308E
:107E6A0000002F00003000002F0000300000380012
:107E7A0000380000383838360000370000E1350095
:107E8A002F00003000001D2F001D30002F00003091
:107E9A0000001D38003800001D370036000037008A
:107EAA0000E13500151210042800110C06122800F2
:107EBA0010171C13082817151211280016170C067C
:107ECA000E281B2327272128062800000000060D5C
:107EDA0028000000060D10040628162800000000DD
:107EEA00160D28000000160D100406282F00003079
:107EFA0000002F00003000002F0000300000380082
:107F0A0000380000383838360000370000E1350004
:107F1A000F28000006280000152800000F2D112840
:107F2A00062D0628152D1628120909281A034500B8
:107F3A007300720069006C006C0065002000490043
:107F4A006E0063002E00181628000018162D072848
:107F5A0018162D06280D132800000D132D112808B8
:107F6A0016150C0F0F082C110C16160828150819CF
:107F7A00372C0007272800071E1F28071F2128075C
:107F8A002023280721252810162800000417120E7E
:107F9A00280A12120A280413130F281201000200D9
:107FAA00000008D80450F50100010200018B00000E
:107FBA008A000088000035000012090928121128D9
:107FCA00000F080728190815372C001304072C007E
:107FDA0009262C0009202C0009212C0009222C003A
:107FEA0009232C0009242C0009252C000E16170B36
:067FFA000403090400006D
:020000040020DA
:08000000FFFFFFFFFFFFFFFF00
:020000040030CA
:0E000000300E3F1EFF8181FF0FC00FE00F404A
:0200000400F00A
:080000000000000100040000F3
:00000001FF
